:100000000C945B000C9483000C9483000C9483008C
:100010000C9483000C9483000C9483000C94830054
:100020000C9483000C9483000C9483000C94830044
:100030000C9483000C9483000C9483000C94830034
:100040000C94C0030C9483000C9441060C94830020
:100050000C9483000C9483000C9483000C94830014
:100060000C9483000C948300000024272A000025B0
:10007000282B000023262904040404040404040299
:100080000202020202030303030303010204081035
:100090002040800102040810200102040810200002
:1000A0000000070002010000030406000000000039
:1000B00000000000180211241FBECFEFD4E0DEBF05
:1000C000CDBF11E0A0E0B1E0E4EDFDE002C005909D
:1000D0000D92AA33B107D9F711E0AAE3B1E001C04C
:1000E0001D92A43DB107E1F710E0C6EBD0E004C0DB
:1000F0002297FE010E94E406C43BD107C9F70E9483
:1001000011020C94E8060C94000040E855E260E00F
:1001100070E086E491E00E942C0264E670E080E0EA
:1001200090E00E942B0461E080911B010E94120567
:1001300061E080911D010E94120561E080911F0124
:100140000E94120560E08EE00E94120560E08FE0E0
:100150000E94120560E080E10E94120560E081E1EA
:100160000E94120561E08EE00E94300561E08FE0A0
:100170000E94300561E080E10E94300561E081E18C
:100180000E94300580913A010E94A0048150924063
:100190003CF081E090E090933D0180933C0104C0ED
:1001A00010923D0110923C01809121010E94A00417
:1001B000815092403CF082E090E090933F01809328
:1001C0003E0104C010923F0110923E018091230134
:1001D0000E94A004815092403CF084E090E0909313
:1001E00041018093400104C01092410110924001EE
:1001F000809125010E94A004815092403CF088E04B
:1002000090E0909343018093420104C01092430117
:100210001092420180913E0190913F0120913C015A
:1002200030913D01820F931F209140013091410197
:10023000820F931F2091420130914301820F931F3F
:10024000909345018093440160E071E086E491E081
:100250000E944102609144017091450186E491E061
:100260000E949003089560E080912F010E94300564
:1002700060E0809131010E94300560E070E0809183
:1002800029010E94BE04089560E080912B010E9424
:10029000300560E080912D010E94300560E070E043
:1002A000809127010E94BE0408950F931F938C0133
:1002B00060E080912F010E94300561E08091310162
:1002C0000E943005B801809129010E94BE041F914F
:1002D0000F9108950F931F938C0161E080912F017E
:1002E0000E94300560E0809131010E943005B80124
:1002F000809129010E94BE041F910F9108950F93D0
:100300001F938C0160E080912B010E94300561E019
:1003100080912D010E943005B801809127010E9433
:10032000BE041F910F9108950F931F938C0161E0FC
:1003300080912B010E94300560E080912D010E9488
:100340003005B801809127010E94BE041F910F91D2
:10035000089586E491E00E942902882309F460C090
:1003600086E491E00E942602909345018093440127
:100370008735910549F48FEF90E00E946A0161E0B2
:1003800080911F010E9430058091440190914501A8
:100390008A35910549F48FEF90E00E94550161E0A4
:1003A00080911F010E943005809144019091450188
:1003B0008134910549F48FEF90E00E94940161E04F
:1003C00080911F010E943005809144019091450168
:1003D0008335910549F48FEF90E00E947F0161E041
:1003E00080911F010E943005809144019091450148
:1003F0008035910539F40E94330160E080911F013E
:100400000E94300580914401909145018F349105FF
:1004100039F40E94440160E080911F010E94300580
:1004200008950E9463040E9485000E94A901FDCFE7
:1004300087E391E090934701809346010895862FCA
:100440000E94000608950E94380608950E94190629
:1004500008950E9408060895CB01BA010E94C705BD
:100460000895DC01ED91FC910190F081E02D09955A
:100470000895DC01ED91FC910190F081E02D09954A
:1004800008950F931F93CF93DF938C01EB0109C065
:100490002196D801ED91FC910190F081E02DC801E9
:1004A000099568816623A1F7DF91CF911F910F9184
:1004B00008950F931F938C01DC01ED91FC91019045
:1004C000F081E02D6DE00995D801ED91FC9101904E
:1004D000F081E02D6AE0C80109951F910F91089500
:1004E0000F931F938C01DC01ED91FC910190F08141
:1004F000E02D0995C8010E9459021F910F9108959E
:100500000F931F938C010E944102C8010E9459025F
:100510001F910F9108950F931F938C01DC01ED91B2
:10052000FC910190F081E02D0995C8010E945902CB
:100530001F910F9108952F923F924F925F926F9269
:100540007F928F929F92AF92BF92CF92DF92EF9263
:10055000FF920F931F93DF93CF93CDB7DEB7A09792
:100560000FB6F894DEBF0FBECDBF1C016A017B0140
:10057000411551056105710549F4DC01ED91FC91CE
:100580000190F081E02D60E3099554C088249924FE
:100590005401422E55246624772401E010E00C0F0C
:1005A0001D1F080D191DC701B601A30192010E946C
:1005B0009106F80160830894811C911CA11CB11C58
:1005C000C701B601A30192010E949106C901DA0197
:1005D0006C017D01C114D104E104F104F1F681E064
:1005E000E82EF12CEC0EFD1EE80CF91C3E010894DF
:1005F000611C711CD501C4010197A109B1096C01ED
:10060000C818D90814C0F601EE0DFF1D60816A30CC
:1006100010F4605D01C0695CD101ED91FC91019025
:10062000F081E02DC10109950894E108F1086E14EC
:100630007F0449F7A0960FB6F894DEBF0FBECDBF7A
:10064000CF91DF911F910F91FF90EF90DF90CF90AE
:10065000BF90AF909F908F907F906F905F904F90E2
:100660003F902F9008952AE00E949B0208950F93D7
:100670001F938C010E943303C8010E9459021F91ED
:100680000F910895AB0160E070E00E94330308957C
:100690000F931F938C01AB0160E070E00E94330365
:1006A000C8010E9459021F910F910895EF92FF9285
:1006B0000F931F93CF93DF93EC017A018B0177FFA8
:1006C0000FC0E881F9810190F081E02D6DE209957C
:1006D00010950095F094E094E11CF11C011D111D92
:1006E0002AE0B801A701CE010E949B02DF91CF91C1
:1006F0001F910F91FF90EF9008950F931F938C011E
:100700000E945603C8010E9459021F910F9108953B
:10071000AB01662757FD6095762F0E94560308951A
:100720000F931F938C01AB01662757FD6095762FC1
:100730000E945603C8010E9459021F910F9108950B
:10074000DC012115310541F4ED91FC910190F0811E
:10075000E02D642F099508952A30310519F40E947F
:10076000560308950E949B0208950F931F938C01D6
:100770000E94A003C8010E9459021F910F91089581
:100780001F920F920FB60F9211242F938F939F9366
:10079000AF93BF938091480190914901A0914A0184
:1007A000B0914B018050904CAF4FBF4F80934801A8
:1007B00090934901A0934A01B0934B0127C08091C7
:1007C000480190914901A0914A01B0914B01805894
:1007D0009E43A040B0408093480190934901A0936C
:1007E0004A01B0934B0180914C0190914D01A09131
:1007F0004E01B0914F010196A11DB11D80934C0196
:1008000090934D01A0934E01B0934F018091480108
:1008100090914901A0914A01B0914B0181589E43AA
:10082000A040B04060F6BF91AF919F918F912F9102
:100830000F900FBE0F901F9018958FB7F8942091CE
:100840004C0130914D0140914E0150914F018FBFAD
:10085000B901CA010895EF92FF920F931F937B0194
:100860008C018FB7F89440914C0150914D016091EB
:100870004E0170914F018FBF2FB7F89480914C01BA
:1008800090914D01A0914E01B0914F012FBF841B5B
:10089000950BA60BB70B8E159F05A007B10760F34C
:1008A0001F910F91FF90EF900895019759F0FC016F
:1008B000EE0FFF1FEE0FFF1F32978FB7F89431979F
:1008C000F1F78FBF0895789484B5826084BD84B5B4
:1008D000816084BD85B5826085BD85B5816085BD3B
:1008E000EEE6F0E0808181608083E1E8F0E08081E5
:1008F00082608083808181608083E0E8F0E0808195
:1009000081608083E1EBF0E0808184608083E0EBB4
:10091000F0E0808181608083EAE7F0E0808184609C
:1009200080838081826080838081816080838081F8
:10093000806880831092C1000895809339010895E2
:100940008F70909139019295990F990F907C982B07
:1009500090937C0080917A00806480937A008091EB
:100960007A0086FDFCCF2091780040917900942F89
:1009700080E030E0282B392BC90108951F93CF93D5
:10098000DF93182FEB0161E00E941205E12FF0E0E8
:10099000E156FF4F8491833051F48091800080684C
:1009A00080938000D0938900C093880037C0843042
:1009B00051F480918000806280938000D0938B00FE
:1009C000C0938A002BC0813029F484B5806884BD2F
:1009D000C7BD24C0823029F484B5806284BDC8BDFF
:1009E0001DC0863041F48091B00080688093B000D3
:1009F000C093B30013C0873041F48091B00080628F
:100A00008093B000C093B40009C0C038D10514F47D
:100A100060E001C061E0812F0E943005DF91CF913D
:100A20001F910895282F30E0C90185579F4FFC0181
:100A3000949129583F4FF9018491882381F0E82F40
:100A4000F0E0E859FF4FE491F0E0662329F480815B
:100A500090958923808308958081892B80830895D0
:100A6000482F50E0CA0181569F4FFC012491CA01D2
:100A700085579F4FFC01949149585F4FFA0134917B
:100A80003323C1F1222331F1233021F480918000FE
:100A90008F7705C0243031F4809180008F7D809362
:100AA000800018C0213019F484B58F7704C022303B
:100AB00021F484B58F7D84BD0DC0263021F4809152
:100AC000B0008F7705C0273029F48091B0008F7D6A
:100AD0008093B000E32FF0E0E359FF4FE491F0E0A2
:100AE000662329F4808190958923808308958081ED
:100AF000892B80830895482F50E0CA0181569F4F6B
:100B0000FC012491CA0185579F4FFC0194914958DB
:100B10005F4FFA013491332319F420E030E035C0FF
:100B2000222331F1233021F4809180008F7705C09A
:100B3000243031F4809180008F7D8093800018C034
:100B4000213019F484B58F7704C0223021F484B5A4
:100B50008F7D84BD0DC0263021F48091B0008F7749
:100B600005C0273029F48091B0008F7D8093B000BC
:100B7000E32FF0E0EE58FF4FE491F0E0808120E0B9
:100B800030E0892311F021E030E0C9010895EF92AF
:100B9000FF920F931F937B018C0122E030E040E035
:100BA00050E00E94B306205C3D4B404F5F4FCA01AE
:100BB000B901A80197010E94B306C901DA010197A2
:100BC000A109B109292F3A2F4B2F552747FD5A95D7
:100BD0000196A11DB11D2093C50081508093C400D2
:100BE000E1ECF0E080818061808380818860808397
:100BF0008081806880831F910F91FF90EF9008950E
:100C0000982F8091C00085FFFCCF9093C600089577
:100C1000809150019091510180589F4F2091520135
:100C200030915301821B930B60E870E00E947E06B6
:100C3000089540915201509153018091500190913B
:100C400051018417950719F42FEF3FEF0FC0FA01F8
:100C5000EC5AFE4F2081CA01019660E870E00E94C4
:100C60007E06909353018093520130E0C9010895AC
:100C700080915201909153019093510180935001C2
:100C800008951F920F920FB60F9211242F933F9346
:100C90004F935F936F937F938F939F93AF93BF9384
:100CA000EF93FF934091C600E0915001F091510104
:100CB000CF01019660E870E00E947E069C01809161
:100CC0005201909153012817390739F0EC5AFE4F21
:100CD00040833093510120935001FF91EF91BF91D8
:100CE000AF919F918F917F916F915F914F913F91C4
:100CF0002F910F900FBE0F901F90189597FB092E04
:100D000007260AD077FD04D049D006D000201AF477
:100D1000709561957F4F0895F6F7909581959F4F57
:100D20000895A1E21A2EAA1BBB1BFD010DC0AA1F2C
:100D3000BB1FEE1FFF1FA217B307E407F50720F044
:100D4000A21BB30BE40BF50B661F771F881F991FBF
:100D50001A9469F760957095809590959B01AC0108
:100D6000BD01CF01089597FB092E05260ED057FD32
:100D700004D0D7DF0AD0001C38F450954095309548
:100D800021953F4F4F4F5F4F0895F6F7909580950F
:100D9000709561957F4F8F4F9F4F0895AA1BBB1B86
:100DA00051E107C0AA1FBB1FA617B70710F0A61B6B
:100DB000B70B881F991F5A95A9F780959095BC018C
:100DC000CD010895EE0FFF1F0590F491E02D0994D9
:040DD000F894FFCFC5
:100DD400486F6C612C20736F7920656C20726F6290
:100DE4006F74206E756D65726F2000060008000B2D
:100DF4000001000200030009000A000200030005CC
:0A0E0400000400000000001F0201BE
:00000001FF
